:10055C0012010002000000400516034001000102D8
:10056C0000010A0600020000004001000902200000
:10057C00010100A0320904000002FF000000070581
:10058C000202000200070586020002000902200098
:10059C00010100A0320904000002FF000000070561
:1005AC000102400000070581024000000403090419
:1005BC00260341004300430045005300200049003E
:1005CC002F004F002000500072006F006400750077
:1005DC0063007400730018035500530042002D0093
:1005EC0044004100310032002D003800450000006D
:03004300020400B4
:03005300020400A4
:100400000209ED00020A7200020A5C00020A4400BE
:1004100002083100020868000200320002004200B7
:10042000020052000203FF00020AD000020AD100BB
:10043000020AD200020AD300020AD400020AD5003E
:10044000020AD60002004200020AD700020AD800BF
:10045000020AD900020ADA00020ADB00020ADC0002
:10046000020ADD00020042000200420002004200D7
:10047000020ADE00020ADF00020AE000020AE100CE
:10048000020AE200020AE300020AE400020AE500AE
:10049000020AE600020AE700020AE800020AE9008E
:1004A000020AEA00020AEB00020AEC00020AED006E
:0804B000020AEE00020AEF004F
:0A0A9A000001020203030404050535
:1005FC00E4F536F535F534F533C203C200C202C258
:10060C0001120036750A05750B5C75120575136EB3
:10061C0075080575097875100575119875140575AB
:10062C0015B8D2E843D82090E668E04409F090E68B
:10063C005CE0443DF0D2AFD20412000390E680E0BF
:10064C0054F7F0538EF8C203300105120056C20164
:10065C00300329120AC45024C2031209C820001600
:10066C0090E682E030E704E020E1EF90E682E030B3
:10067C00E604E020E0E4120970120AC612071980A1
:01068C00C7A6
:1000560090E6B9E0700302010714700302018424DC
:10006600FE700302020724FB7003020101147003F1
:100076000200FB14607314607624056003020266B6
:10008600120AC8400302027290E6BBE024FE602218
:1000960014603324FD601114602224067048E50ABA
:1000A60090E6B3F0E50B8037E51290E6B3F0E51382
:1000B600802DE50C90E6B3F0E50D8023E50E90E685
:1000C600B3F0E50F801990E6BAE0FF12099CAA0684
:1000D600A9077B01EA494B600DEE90E6B3F0EF907D
:1000E600E6B4F002027202026B120A88020272126F
:1000F6000AAC020272120AA40202721203ED020292
:1001060072120ACA400302027290E6B8E0247F60C7
:100116001514601924027063A200E43325E0FFA2DF
:1001260002E4334F8041E490E740F0803F90E6BC24
:10013600E0547EFF7E00E0D394807C0040047D0185
:1001460080027D00EC4EFEED4F249AF582740A3E45
:10015600F583E493FF3395E0FEEF24A1FFEE34E64A
:100166008F82F583E0540190E740F0E4A3F090E637
:100176008AF090E68B7402F002027202026B120A97
:10018600CC400302027290E6B8E024FE6016240218
:10019600600302027290E6BAE0B40105C2000202F0
:1001A6007202026B90E6BAE0705590E6BCE0547EAF
:1001B600FF7E00E0D394807C0040047D0180027DB8
:1001C60000EC4EFEED4F249AF582740A3EF583E468
:1001D60093FF3395E0FEEF24A1FFEE34E68F82F520
:1001E60083E054FEF090E6BCE05480131313541FD2
:1001F600FFE0540F2F90E683F0E04420F0806D80FE
:1002060064120ACE506690E6B8E024FE6019240215
:10021600705A90E6BAE0B40104D200804F90E6BA74
:10022600E064026047803E90E6BCE0547EFF7E00BC
:10023600E0D394807C0040047D0180027D00EC4E7A
:10024600FEED4F249AF582740A3EF583E493FF335C
:1002560095E0FEEF24A1FFEE34E68F82F583800859
:10026600120382500790E6A0E04401F090E6A0E079
:030276004480F0D1
:010279002262
:0300330002004E7A
:04004E0053D8EF3262
:04004600021600009E
:0C003600D200120AB4E4F5B175B63F2206
:040ABC0043B1202200
:040AC00053B1DF222D
:10071900E51A6035E5174516700675162F7517FF2A
:10072900E517151770021516E51745167004F51A21
:10073900800FAE16AF177C0B7DFF120507EF20E087
:1007490005120AC08003120ABCE5B190E68020E7D1
:0A07590005E04408F022E054F7F038
:010763002273
:020AC400D3223B
:020AC600D32239
:020AC800D32237
:080AA40090E6BAE0F51BD32235
:1003ED0090E740E51BF0E490E68AF090E68B04F090
:0203FD00D32209
:080AAC0090E6BAE0F518D32230
:100A880090E740E518F0E490E68AF090E68B04F0F1
:020A9800D32267
:020ACA00D32235
:020ACC00D32233
:020ACE00D32231
:10038200751A0190E678E05410C4540F4450F519E0
:1003920013E433F51C90E6B9E0244D704A90E6BEB2
:1003A200E090E68BF090E6A0E020E1F990E6BEE076
:1003B200D39400503490E6BAE0FF90E6BCE075F0CA
:1003C20002A42400F582E5F03480F583EFF090E694
:1003D200BBE0FFA3E075F002A42401F582E5F0344E
:0B03E20080F583EFF08002D322C322DD
:1009ED00C0E0C083C08290E6B5E04401F0D201536F
:0F09FD0091EF90E65D7401F0D082D083D0E032AC
:100A5C00C0E0C083C0825391EF90E65D7404F0D087
:060A6C0082D083D0E032CD
:100A7200C0E0C083C0825391EF90E65D7402F0D073
:060A820082D083D0E032B7
:10083100C0E0C083C08290E680E030E70E85080CFE
:1008410085090D85100E85110F800C85100C851101
:100851000D85080E85090F5391EF90E65D7410F038
:07086100D082D083D0E03209
:100A4400C0E0C083C082D2035391EF90E65D740886
:080A5400F0D082D083D0E03223
:10086800C0E0C083C08290E680E030E70E85080CC7
:1008780085090D85100E85110F800C85100C8511CA
:100888000D85080E85090F5391EF90E65D7420F0F1
:07089800D082D083D0E032D2
:01003200329B
:01004200328B
:01005200327B
:0103FF0032CB
:010AD00032F3
:010AD10032F2
:010AD20032F1
:010AD30032F0
:010AD40032EF
:010AD50032EE
:010AD60032ED
:010AD70032EC
:010AD80032EB
:010AD90032EA
:010ADA0032E9
:010ADB0032E8
:010ADC0032E7
:010ADD0032E6
:010ADE0032E5
:010ADF0032E4
:010AE00032E3
:010AE10032E2
:010AE20032E1
:010AE30032E0
:010AE40032DF
:010AE50032DE
:010AE60032DD
:010AE70032DC
:010AE80032DB
:010AE90032DA
:010AEA0032D9
:010AEB0032D8
:010AEC0032D7
:010AED0032D6
:010AEE0032D5
:010AEF0032D4
:0407F200AA06AC05A2
:1007F600E4FD7E000DEE2400F582E43400F583EA84
:10080600F00E0D74002EF582E43400F583EFF00D42
:1008160074002402F582E43400F583ECF07A007B60
:0B08260000AF19120A28AF1902089F4A
:0A08D5008E218F228D238A248B25AB
:1008DF00E4F526E526C3952350200522E522AE2117
:1008EF007002052114FFE5252526F582E43524F550
:0A08FF0083E0FD1207F2052680D900
:0109090022CB
:0A0764008E278F288D298A2A8B2BFF
:10076E00E4FDF52CE51C6012E527FF7E000DEE245E
:10077E0003F582E43400F583EFF0AE050D74032E1D
:10078E00F582E43400F583E528F07A007B03AF1997
:0E079E00120A28AB2BAA2AAD29AF19020A0CA9
:1009700090E682E030E004E020E60B90E682E03092
:10098000E119E030E71590E680E04401F07F147E45
:0C099000001207AC90E680E054FEF0225C
:1009C80090E682E044C0F090E681F04387010000A1
:0409D80000000022F9
:1000030030040990E680E0440AF0800790E680E03F
:100013004408F07FDC7E051207AC90E65D74FFF0C8
:0F00230090E65FF05391EF90E680E054F7F02203
:080AB400E4F532D2E9D2AF22D1
:10089F0090E678E020E6F9C2E990E678E04480F04F
:1008AF00EF25E090E679F090E678E030E0F990E619
:1008BF0078E04440F090E678E020E6F990E678E0C2
:0608CF0030E1D6D2E9225F
:10093E00A90790E678E020E6F9E532702390E67894
:10094E00E04480F0E925E090E679F08D2DAF03A923
:10095E0007752E018A2F8930E4F531753201D322C5
:02096E00C322A2
:10090A00A90790E678E020E6F9E532702590E678C6
:10091A00E04480F0E925E0440190E679F08D2DAFBE
:10092A0003A907752E018A2F8930E4F53175320340
:04093A00D322C322DF
:03004B0002027A34
:10027A00C0E0C083C082C085C084C086758600C0C5
:10028A00D075D000C000C001C002C003C006C007BC
:10029A0090E678E030E20675320602036490E6786A
:1002AA00E020E10CE532640260067532070203645D
:1002BA00E53224FE605F14603624FE7003020355A3
:1002CA0024FC700302036124086003020364AB2E5A
:1002DA00AA2FA930AF3105318F827583001204B875
:1002EA0090E679F0E531652D7070753205806B9076
:1002FA00E679E0AB2EAA2FA930AE318E8275830043
:10030A001204E5753202E52D6401704E90E678E03C
:10031A004420F08045E52D24FEB5310790E678E0CB
:10032A004420F0E52D14B5310A90E678E04440F017
:10033A0075320090E679E0AB2EAA2FA930AE318E45
:10034A00827583001204E50531800F90E678E04457
:10035A0040F075320080037532005391DFD007D028
:10036A0006D003D002D001D000D0D0D086D084D01D
:08037A0085D082D083D0E0326F
:02099C00A907A9
:10099E00AE14AF158F828E83A3E064037017AD0182
:1009AE0019ED7001228F828E83E07C002FFDEC3ECC
:0909BE00FEAF0580DF7E007F0022
:0109C700220D
:100A0C0012090AE53224FA600E146006240770F30A
:0C0A1C00D322E4F532D322E4F532D322D9
:100A280012093EE53224FA600E146006240770F3BA
:0C0A3800D322E4F532D322E4F532D322BD
:1007AC008E378F3890E600E054187012E53824012B
:1007BC00FFE43537C313F537EF13F538801590E6A2
:1007CC0000E05418FFBF100BE53825E0F538E5378D
:1007DC0033F537E5381538AE37700215374E6005EE
:0607EC001209DC80EE2280
:1009DC007400F58690FDA57C05A3E582458370F92E
:0109EC0022E8
:0300000002068D68
:0C068D00787FE4F6D8FD7581380206D4B1
:1004B800BB010CE58229F582E5833AF583E02250F9
:1004C80006E92582F8E622BBFE06E92582F8E22243
:0D04D800E58229F582E5833AF583E493225D
:1004E500F8BB010DE58229F582E5833AF583E8F04D
:1004F500225006E92582C8F622BBFE05E92582C8F9
:02050500F222E0
:10050700BC000BBE0029EF8DF084FFADF022E4CCD8
:10051700F875F008EF2FFFEE33FEEC33FCEE9DECA1
:10052700984005FCEE9DFE0FD5F0E9E4CEFD22EDE7
:10053700F8F5F0EE8420D21CFEADF075F008EF2F31
:10054700FFED33FD4007985006D5F0F222C398FD22
:050557000FD5F0EA22BF
:100699000205FCE493A3F8E493A34003F68001F276
:1006A90008DFF48029E493A3F85407240CC8C33362
:1006B900C4540F4420C8834004F456800146F6DF31
:1006C900E4800B0102040810204080900046E47E7B
:1006D900019360BCA3FF543F30E509541FFEE49326
:1006E900A360010ECF54C025E060A840B8E493A3ED
:1006F900FAE493A3F8E493A3C8C582C8CAC583CA18
:10070900F0A3C8C582C8CAC583CADFE9DEE780BECF
:01004A0000B5
:00000001FF
